:1000000000060020250B0000110400005509000027
:1000100000000000000000000000000000000000E0
:100020000000000000000000000000005509000072
:10003000000000000000000055090000310700002A
:1000400000000000000000000000000000000000B0
:100050000000000055090000550900005509000086
:100060005509000000000000550900005509000076
:1000700055090000950700005509000055090000CA
:1000800055090000550900005509000055090000F8
:1000900055090000550900005509000055090000E8
:1000A0005509000055090000000000005509000036
:1000B00055090000000000000000000000000000E2
:10040000FFFFFFFFFFFFFFFFFFFFFFFF80E442FF53
:100410000822014B5A607047008004400022014BC3
:100420001A707047D0020020F7B5B24C002526782C
:10043000012E49D16378AB4228D163792579022016
:10044000ED18E37A0335ED18A37AED18637AED1809
:10045000237AED1800F018FA300000F015FA207930
:1004600000F012FA607900F00FFAE07A00F00CFA6E
:10047000A07A00F009FA607A00F006FAEDB2207A6C
:1004800000F002FA280000F0FFF909E0012B07D183
:1004900023000C33E85C013500F0F6F9092DF7D1A3
:1004A000002323706370637D002B01D00123A375AB
:1004B0006B46DD1D280000F001FA002823D102223E
:1004C000237893435BD1F7BD022EE9D10127300099
:1004D000A780A56000F0D8F9380000F0D5F92079A0
:1004E00000F0D2F9607900F0CFF9E07A00F0CCF9B1
:1004F000A07A00F0C9F9607A00F0C6F9207A00F01D
:10050000C3F90420BFE700F0F7F9002801D0002369
:10051000E375E27D2978531CDBB2A218E3751176EE
:10052000092BCCD10023227EE375012AC7D12000FC
:100530001A001830195C01335218D2B2082BF9D1C5
:10054000631CDB7F934229D1627E631DDA77A27E32
:10055000A31DDA77E27EE31DDA772300227F0C33D6
:10056000DA772300627F0B33DA772300A27F0A3326
:10057000DA772300E27F0933DA77012323706423DB
:10058000621DD07FA16A60712371A160D02816D846
:10059000C72806D8882820D002237DE002232370B4
:1005A00091E7C8380828F7D800F046FA2E003B003B
:1005B00047006800780083008600F6FF9500F22867
:1005C000EAD1626A4C4B13404C4A934263D14C4B84
:1005D000994260D10223637075E7A31DDB7F002B76
:1005E0000CD10121617049182173464C0732185D06
:1005F000991801334870082BF9D164E7012B00D01A
:1006000061E7414BA3605EE7A02480256401ED0112
:1006100020003E4B984780239B00E418AC42F7D162
:1006200051E7E31DDB7FA21DD27F1B029B187F2BAE
:1006300057DC374A9B00995045E7364BC918364B73
:10064000994218D880260025B600A36AE818334BD3
:10065000984203D82E4B5959314B98470435B5422F
:10066000F3D1012000232A4940429A0001338850E7
:10067000802BFAD127E704232371F2E7294B994213
:1006800009DC0022E36A8B4201D9A2601BE71878DB
:1006900001331218F7E70423237114E7E36A8B424E
:1006A000F9D88023DB019942F5D28B07F3D10B688F
:1006B000A8E70123637506E7A31DDB7F012B06D0A6
:1006C000022B06D0002B0CD180239B009AE7E36A13
:1006D00098E7154B96E7A31DDB7F002B03D0012B7A
:1006E00005D00323D8E70F480D4B9847EBE60F489A
:1006F000FAE7C046D002002000FFFF000081920010
:10070000D6C5B4A3F81300000601EA103502002094
:100710000003002000ECFFFFF72B0000F73F000074
:1007200075020020F83F0000F83D0000FC3F00008B
:100730000C4A1368013313600B4B1A68002A08D067
:100740001A68013A1A601B68002B02D10122074B7C
:100750001A70074B1A68002A02D01A68013A1A6008
:100760007047C046000500204C05002048050020C9
:1007700050050020FA22034BD2015A6007221A606A
:100780007047C04610E000E0014B18687047C04653
:100790000005002030B5204B1A79D1B2920614D54D
:1007A0001E4A1468601C092C00D100205468844241
:1007B00005D01468DD791419EDB225721060052496
:1007C000174804605069174A10604020014202D067
:1007D000DA788243DA7049B2002918DA114A1068CF
:1007E000002814D10D4A9469D1698C4210D0D46983
:1007F000611CD161511C0919C97FC9B2D971D16974
:100800000A2900D1D0614022D9780A43DA7030BD7C
:100810007F21DA780A40F9E700B00640040500209D
:100820004C050020500500208023134A9B03D1680B
:1008300010B50B43D3600023104CE370A370A37179
:100840006371072800D918000D4B8000C1580D4B6B
:100850004808C01800F0FAF81F212278030A0B405C
:100860008A43134323702C23C0B260700D20E370C1
:1008700000F08EF810BDC0460080044000B0064075
:100880005C0D000040420F000A4B10B599694A1CEC
:10089000092900D10022D969914209D09C69591CCB
:1008A0000919C87780219A61034AD3780B43D37022
:1008B00010BDC0460405002000B006400A4B10B52C
:1008C0005C681A680100002094420BD05A68501CE2
:1008D00058609A18127A01200A705A680A2A01D1BF
:1008E00000225A6010BDC04604050020014B58612B
:1008F0007047C046040500200020034B1A7882424E
:1009000001D01870013070474805002062B670476A
:1009100072B67047024A034B0349D1507047C04634
:1009200000E000E00C0D00000400FA050E22074B69
:1009300059691143596199680A439A608023044AAE
:10094000DB0351680B4353607047C04600F00F4013
:100950000090044000BE70470749084A084BD15038
:10096000084B094A5A80094A5A809A8000225A70D4
:1009700020321A707047C0460000000000E000E01E
:10098000080D000000200540C5200000D928000007
:10099000202801DDC0467047074B184004D52023AE
:1009A00001385B42184301300123C0218340034AD0
:1009B000490053501360EEE71F00008000E100E0A3
:1009C000202801DDC0467047064B184004D520237F
:1009D00001385B421843013001238340024AD36748
:1009E000F1E7C0461F00008004E100E0020010B5FE
:1009F00020281BDC032919DC0320D31703409B1894
:100A0000FC309B1089010340094C014009489B00C0
:100A10001B19104004D50422013852421043013002
:100A2000C0B2C00081401A681143196010BDC046B1
:100A300000E400E00300008003B471464908400070
:100A40004900095E49008E4403BC7047002934D038
:100A50000123002210B488422CD301242407A14290
:100A600004D2814202D209011B01F8E7E400A1424D
:100A700004D2814202D249005B00F8E7884201D3E8
:100A8000401A1A434C08A04202D3001B5C082243C0
:100A90008C08A04202D3001B9C082243CC08A04231
:100AA00002D3001BDC082243002803D01B0901D01D
:100AB0000909E3E7101C10BC704701B5002000F0E5
:100AC0000BF802BD0029F8D003B5FFF7C1FF0EBC3B
:100AD0004243891A1847C0467047C04610B5064CB5
:100AE0002378002B07D1054B002B02D0044800E0EF
:100AF00000BF0123237010BD2E0500200000000060
:100B0000800D0000044B10B5002B03D003490448AE
:100B100000E000BF10BDC04600000000300500200E
:100B2000800D0000002103E00B4B5B584350043163
:100B30000A480B4B42189A42F6D30A4A02E00023B5
:100B400013600432084B9A42F9D3FFF705FF00F017
:100B50000DF8804770470000A40D000008FEFF1F3D
:100B6000D0020020D002002078050020A02370B51C
:100B70002C4D2D4C2D4A29685B01E362914203D133
:100B80002B4A1268520518D41B68013B033314D852
:100B9000284B19684B1E03330FD80023A0261A00D8
:100BA0007601905D01321B189142FAD1224A1268F7
:100BB0009A4202D1214B186870BD012200260421FF
:100BC0001B4B9A611E4A5670117008225A601D4BC9
:100BD00007321A70197831320A431A70FFF796FEFD
:100BE000FFF7A4FEFFF7C6FD0720FFF71DFE30004C
:100BF000FFF77CFE2670FFF717FC637D002BFAD011
:100C0000A37D002BF7D0FFF783FE00230E4A0F4988
:100C1000136001225242CA67C0210D484900425068
:100C20002B60C7E700FEFF1FD00200207856341269
:100C300000800440F83F0000FC3F00000414000066
:100C4000004006400000024010E000E004E100E047
:100C500000E100E010B5010000230022002000F0B8
:100C600015F810BD70B5074D074C641BA41005D0D6
:100C7000013CA300EB589847002CF9D100F086F80E
:100C800070BDC046A00D0000A40D0000F0B5D64612
:100C90004F464646C0B5274F82B006003868914699
:100CA00098468A4600F056F8234B1B680193A4230C
:100CB000019A5B00D558002D31D06C6838681F2C24
:100CC00032DC002E0ED1631C6B6053460234A4004C
:100CD000635100F041F8002002B01CBC90469946D8
:100CE000A246F0BD88224946A300EB189950C421C2
:100CF00049008C46AC446146873AA2406746096881
:100D0000114339608421474649005F50022EDAD1F1
:100D10002B008D33FF3319680A431A60D3E715009F
:100D20004D35FF35D550C8E700F016F80120404298
:100D3000D2E7C046300200207C0D0000034B10B506
:100D4000002B02D00248FFF785FF10BD0000000015
:100D5000650C00007047C0467047C0468025000003
:100D600040380000004B000080700000009600003A
:100D700000E10000002C010000C2010008FEFF1F7E
:100D8000F8B5C046F8BC08BC9E467047F8B5C046EA
:080D9000F8BC08BC9E46704748
:080D98003D0D0000050B0000F9
:040DA000DD0A000068
:100DA40000000000F40000205C010020C4010020C9
:100DB400000000000000000000000000000000002F
:100DC400000000000000000000000000000000001F
:100DD400000000000000000000000000000000000F
:100DE40000000000000000000000000000000000FF
:100DF40000000000000000000000000000000000EF
:100E040000000000000000000000000000000000DE
:100E140000000000000000000000000000000000CE
:100E240000000000000000000000000000000000BE
:100E340000000000000000000000000000000000AE
:100E4400000000000000000001000000000000009D
:100E54000E33CDAB34126DE6ECDE05000B00000062
:100E6400000000000000000000000000000000007E
:100E7400000000000000000000000000000000006E
:100E8400000000000000000000000000000000005E
:100E9400000000000000000000000000000000004E
:1011C40000000000000000005405002072B6302228
:1011D4000D4B9A719A7952B2002AFBDA00229A7066
:1011E4000A329A72020CD2B2DA7201229A70020A9C
:1011F400D2B29A728022C0B2D8729A719A7952B2DB
:10120400002AFBDA62B670470000024072B6302250
:10121400144B9A719A7952B2002AFBDA00229A701E
:1012240006329A72020CD2B2DA7201229A70020A5F
:10123400D2B29A720222C0B2D8729A700A0AD2B298
:101244009A72CAB2DA7203229A700A0E9A728022D1
:10125400090CC9B2D9729A719A7952B2002AFBDA8E
:0812640062B670470000024071
:10126C00A40D000008FEFF1FC804000000000000D1
:08127C0000000000000000006A
:0813F80032333030423130364F
:020000041FFFDC
:04FE000000000000FE
:0400000300000B25C9
:00000001FF
